:020000040800F2
:10000000304A00204D010008C1180008B110000856
:10001000BD180008C3020008412C000800000000C1
:100020000000000000000000000000006B1C000841
:100030007D0A000800000000630100081D1E000882
:1000400067010008670100086701000867010008F0
:1000500067010008670100086701000867010008E0
:1000600067010008670100086701000867010008D0
:10007000790A0008670100087B0A00086701000888
:1000800067010008670100086701000867010008B0
:1000900067010008670100086701000867010008A0
:1000A0006701000867010008670100086701000890
:1000B0006701000867010008670100086701000880
:1000C0006701000867010008670100086701000870
:1000D00067010008BD270008C5270008CD270008D4
:1000E0006701000867010008670100086701000850
:1000F0006701000867010008670100086701000840
:10010000670100086701000867010008670100082F
:10011000670100086701000867010008670100081F
:10012000670100086701000867010008670100080F
:10013000DFF80CD000F094F800480047A93300081D
:10014000304A002080F30888704700000648804746
:1001500006480047FEE7FEE7FEE7FEE7FEE7FEE7AC
:10016000FEE7FEE7FEE7FEE7891E00083101000812
:1001700040EA01039B0703D009E008C9121F08C029
:10018000042AFAD203E011F8013B00F8013B521EA9
:10019000F9D27047D2B201E000F8012B491EFBD220
:1001A00070470022F6E710B513460A460446194682
:1001B000FFF7F0FF204610BD421E12F8013F002B52
:1001C000FBD111F8013B02F8013B002BF9D170473C
:1001D00010B5002200E0521C835C8C5CA34201D16C
:1001E000002BF8D1D8B2E1B2401A10BD034611F885
:1001F000012B00F8012B002AF9D1184670472DE990
:10020000F05F0546002092469B468846064681469A
:1002100040241BE0284641464746224600F041F86C
:1002200053465A46C01A914110D3114618462246E9
:1002300000F028F82D1A67EB01084F4622460120EE
:10024000002100F01FF817EB00094E41201EA4F119
:100250000104DFDC484631462A464346BDE8F09FAC
:10026000064C074D06E0E06840F0010394E8070003
:1002700098471034AC42F6D3FFF75EFF9839000878
:10028000B8390008202A04DB203A00FA02F10020E5
:1002900070479140C2F1200320FA03F319439040C4
:1002A0007047202A04DB203A21FA02F0002170472F
:1002B00021FA02F3D040C2F12002914008431946CE
:1002C000704700BFFEE7000010B500241548006825
:1002D00000F0080068B100BF13A001F0FDF80A208B
:1002E00000F0CDFB4FF480700E490C31086000BF68
:1002F000FEE70DE0601C04460F49884208D30FA0BA
:1003000001F0EAF84FF4807006490831086010BD2A
:100310000448006800F008000028EBD00AA001F0B3
:10032000DBF8D9E7080C01400D0A5077724F6E4692
:1003300061696C6564000000400D03000D0A507790
:10034000724F6E4F6B0000000D0A5077722065727D
:10035000726F00002DE9F0414FF000082E49496806
:10036000491E01EB410202EBC1022B49083101EBAE
:1003700082002AA1FFF72CFF10B14FF0010810E016
:1003800025484068401E00EB400101EBC0012248B7
:10039000083000EB8100406AB0F5805F01D94FF072
:1003A0000208B8F1000F08D006E01EA001F094F892
:1003B0004FF4FA7000F063FBF7E7002628E01648D8
:1003C0004068401E00EB400101EBC00112480830BC
:1003D00000EB8100846A4FF4FF151EB904F58054C8
:1003E00005F58055002710E04FF480622146124841
:1003F00003F07AF84FF4806229460F4803F0EAF8D8
:1004000004F5806405F580657F1C042FECD3761C11
:10041000022ED4D3BDE8F081AA2600207379732E72
:10042000696E69007379732E696E69206572722C2A
:100430002073746F700D0A00AA2200202DE9F0418C
:1004400004460D46164633462A462146044801F026
:10045000AFF907463946024802F0DCFBBDE8F081FF
:100460009221002010B5044801F0D4F90446214639
:10047000014802F0CFFB10BD922100202DE9F04F82
:1004800091B007460297029F3868FE49884204D01F
:100490004FF0FF3011B0BDE8F08F02980079952839
:1004A00002D06FF00100F5E70298407910900298B1
:1004B000008B0F90109803287ED140F682710F9820
:1004C000884202D06FF00300E4E73D46B5F89ABFDA
:1004D0004FF4786205F11A01002002F0EFFE824627
:1004E000DA4502D06FF00400D4E7D5F81E0008B951
:1004F0000020CFE705F11A0001F0EEFA05F11A002D
:1005000000F084FCE0490880D5F81E000988884284
:1005100009D8D5F81E00DD494860DD48086000F0C4
:1005200073FC0020B6E7D5F81E00D8494860D648CD
:1005300004888EE054B9002104EB440000EBC402AF
:10054000D248083000EB8200816245E0601E00EB7B
:10055000400101EBC001CD48083000EB8100808CE8
:10056000C0F30B09601E00EB400101EBC001C7485E
:10057000083000EB8100806A00F58050611E01EBBD
:10058000410202EBC102C149083101EB8201496A13
:10059000014404EB440000EBC402BC48083000EB0B
:1005A00082008162B9F1000F16D004EB440000EB29
:1005B000C401B648083000E088E000EB8100806AA2
:1005C000C9F58051014404EB440000EBC402AF487C
:1005D000083000EB8200816204EB440000EBC401B0
:1005E00005F1220000EB8100416A04EB440000EBBE
:1005F000C402A648083000EB8200416204EB4402CA
:1006000002EBC40305F1220202EB830202F11401A2
:1006100004EB440202EBC4039C4A083202EB83025F
:1006200002F114001022FFF7A3FD04EB440202EBD9
:10063000C40305F1220202EB830104EB440202EB46
:10064000C403924A083202EB83001422FFF790FDA4
:10065000641C8E484068A0423FF66CAF00208D4974
:1006600008608A4842688CA1904802F0CDFB8F4810
:1006700000F032FF8448008800EB400101EBC0012C
:100680008248083000EB8100406A00907E48008874
:1006900000EB400101EBC0017C48083000EB810316
:1006A00083487949098830F8112082A17F4802F0F7
:1006B000ABFB7E4800F010FF4FF480527548016894
:1006C00071480088FFF7BAFE0120E3E6109804287D
:1006D0007DD13E46D6F83E106B48008800EB4002C4
:1006E00002EBC0026948083000EB8200406A814298
:1006F0000DD1B06C67490968884208D16C486249DD
:10070000098830F81100B6F8461088420DD06FA065
:1007100000F0E2FE4FF480525E4801685A480088BB
:10072000FFF78CFE6FF00500B4E6D6F84C80A8F118
:100730000208424606F15001002002F0BFFD834648
:1007400006F1500008F10101405C4FEA002A06F171
:10075000500010F8080050441FFA80FADA450DD016
:1007600061A000F0B9FE4FF480524A480168464843
:100770000088FFF763FE6FF007008BE61FFA88F230
:100780004148008800EB400303EBC0033F480830BA
:1007900000EB8300806A00F580503E4B1B68C11857
:1007A00006F1500002F016FF3A48006808EB00011D
:1007B000D6F83E00814263D33348008800F04CFAFB
:1007C00078BB0020334908602F48008800E031E101
:1007D00000EB400101EBC0012C48083000EB810028
:1007E000406A00902848008800EB400101EBC001FE
:1007F0002648083000EB81032D482349098830F84A
:1008000011202CA1294802F0FFFA284800F064FECC
:100810004FF480521F4801681B480088FFF70EFE06
:1008200006E1FFE71848008800EB400101EBC0013A
:100830001648083000EB8100406A0C90124800888E
:1008400000EB400202EBC0021048083000EB8201CE
:10085000142203A8FFF78CFC0B48008800EB400231
:1008600002EBC0020948083000EB820000F11401DD
:10087000102208A8FFF77CFC1F480E9002483DE0BC
:10088000AEE0000050435441B4000020AA260020EE
:10089000F8DEBC8AB80000205246696C6520436FC0
:1008A000756E743D256C750D0A000000AA220020AB
:1008B000F62100205246696C655B25645D3A25731C
:1008C000206C656E3D256C750D0A0000464C656E0A
:1008D000206F72204F6666736574206572722152B4
:1008E00065444F210D0A0000435243206572722176
:1008F0005265444F210D0A00311B2008008810B9B1
:1009000000200D900AE04C48008800EB400101EB0C
:10091000C0014A4800EB8100806A0D900C98C0F33A
:100920000B09DDE90C0100F5805008440D90B9F188
:10093000000F04D0C9F580510D9808440D903F4830
:10094000083841683C480088401C814201D800209A
:100950000D903948008800EB400202EBC002374896
:1009600000EB8200816A302203A802F033FE324895
:100970000088401C80B230490880304908394968F5
:10098000884201D3002085E500202D4908602A48CF
:10099000008800EB400101EBC001284800EB81001A
:1009A000406A00902448008800EB400101EBC00140
:1009B000224800EB810323481F49098830F81120A1
:1009C00021A1274802F020FA254800F085FD4FF4C8
:1009D00080521B48016818480088FFF72FFD27E068
:1009E00017480068404416490860084600686421BA
:1009F00048431149098801EB410202EBC1020F494A
:100A000001EB8201496AB0FBF1F0034601900C480A
:100A100014A10268124802F0F7F9114800F05CFDD9
:100A20004FF480520648016803480088FFF706FD2E
:100A300002202FE500BF2DE5B4000020B2260020E3
:100A4000B8000020F62100205246696C655B2564E1
:100A50005D3A257320206C656E3D256C750D0A008E
:100A6000AA2200206F66667365743D2564202564A4
:100A700025250D0A0000000070477047704710B52B
:100A8000024607E0002101E04B1C99B241F270736D
:100A90009942F9DB131EA2F10104A2B2F2D110BDFA
:100AA0004FF0E0231A6900210CE008E04FF0E0234A
:100AB0001B69934203D04FF0E0231A6900E0F5E789
:100AC00000BF491C8142F0DB704701461CE000BFBB
:100AD00000BF00BF00BF00BF00BF00BF00BF00BF1E
:100AE00000BF00BF00BF00BF00BF00BF00BF00BF0E
:100AF00000BF00BF00BF00BF00BF00BF00BF00BFFE
:100B000000BF00BF00BF00BF0A1EA1F1010399B2E0
:100B1000DDD170470149C8607047000000200240E5
:100B200030B5044604254FF4302000F082F8054625
:100B3000042D17D10C48006940F002000A490861F1
:100B400008464461006940F0400008614FF43020DD
:100B500000F06FF805460448006941F6FD71084051
:100B600001490861284630BD0020024004200B499D
:100B7000C96801F0010109B101200EE00749C96807
:100B800001F0040109B1022007E00449C96801F03D
:100B9000100109B1032000E004207047002002404A
:100BA0000348006940F08000014908617047000077
:100BB0000020024070B504460D460426F00200F005
:100BC00038F80646042E11D10948006940F00100AA
:100BD000074908612580F00200F02BF8064604481A
:100BE000006941F6FE71084001490861304670BD58
:100BF00000200240024803494860034848607047AB
:100C00002301674500200240AB89EFCD00B50246C5
:100C10000423FFF7ABFF034603E0FFF7A7FF0346FC
:100C2000521E012B01D1002AF7D102B90523184623
:100C300000BD00B502460423FFF798FF034603E01A
:100C4000FFF794FF0346521E012B01D1002AF7D172
:100C500002B90523184600BD2DE9F043ADF26C4DF5
:100C6000064606EB460000EBC6012B4800EB810070
:100C7000D0F8249006EB460000EBC601264800EBB6
:100C80008100876A07F58057B8464D460DF204404B
:100C900000F0C6FC20E0B5F5806F11D94FF48062FA
:100CA000414601A802F020FC4FF4806201A90DF238
:100CB000044000F0C7FC08F58068A5F580650BE0EE
:100CC000AAB2414601A802F00FFC2A4601A90DF282
:100CD000044000F0B7FC0025002DDCD10DF20440EB
:100CE00000F036FC002413E006EB460000EBC601E2
:100CF000094800EB81001430015D0DF25C40005D9D
:100D0000814204D000200DF26C4DBDE8F083641CDC
:100D1000102CE9DB0120F6E7B226002010B500F028
:100D200017F809480068094988420BD04FF47861E8
:100D30000548FFF736FA05480349086000F064F8F3
:100D4000012010BD0020FCE7AA260020F8DEBC8AA6
:100D500030B58DB04FF478612748FFF722FA0024B0
:100D600000253DE03022294601A802F0BDFB2349C1
:100D70000C98884232D104EB440101EBC4021E49B5
:100D8000083101EB8200142201A9FFF7F1F904EB0D
:100D9000440101EBC4021849083101EB820101F161
:100DA0001400102206A9FFF7E3F904EB440000EB5E
:100DB000C4021148083000EB82000A99416204EB3A
:100DC000440000EBC4010C48083000EB8100856250
:100DD000641C0B9808B10B9D02E004E005F58055FA
:100DE00007488542BEDB00BF0348446014B1054894
:100DF000014908600DB030BDAA260020311B200833
:100E0000FFDF1F00F8DEBC8A7047000070B50646A1
:100E1000002446E004EB440000EBC401254800EB4D
:100E20008100416A04EB440000EBC40206F10800B3
:100E300000EB8200406A814200D037E0002516E0D6
:100E400004EB440000EBC4011A4800EB81001430AD
:100E5000415D04EB440000EBC40206F1080000EB26
:100E600082001430405D814200D002E06D1C102DE4
:100E7000E6DB00BF102D00D018E004EB440202EBCB
:100E8000C40306F1080202EB830104EB440202EB07
:100E9000C403084A02EB8300FFF79AF900B105E0AA
:100EA000641C044808384068A042B3D800BF2046FC
:100EB00070BD0000B22600202DE9F0410246002559
:100EC0000026002000230024002791F803C00CF026
:100ED0000F0591F803C00CF0100CBCF1000F03D00B
:100EE00091F802C04CEA050591F800C0BCF1000F72
:100EF00031D0146800202BE04FF0010C0CFA00F305
:100F0000B1F800C00CEA03069E4220D183004FF0E6
:100F10000F0C0CFA03F7BC4305FA03FC4CEA04047B
:100F200091F803C0BCF1280F06D14FF0010C0CFA68
:100F300000FCC2F814C00AE091F803C0BCF1480FED
:100F400005D14FF0010C0CFA00FCC2F810C0401C97
:100F50000828D1D31460B1F800C0BCF1FF0F34DD14
:100F6000546800202EE000F1080C4FF0010808FA48
:100F70000CF3B1F800C00CEA03069E4221D18300B5
:100F80004FF00F0C0CFA03F7BC4305FA03FC4CEAD4
:100F9000040491F803C0BCF1280F05D100F1080C3E
:100FA00008FA0CF8C2F8148091F803C0BCF1480F9D
:100FB00007D100F1080C4FF0010808FA0CF8C2F84C
:100FC0001080401C0828CED35460BDE8F08100009A
:100FD000F0B50A46002300240021002500F0004659
:100FE000B6F1004F02D11D4EF16901E01B4E716850
:100FF000C0F3034583B200F44016B6F5401F08D194
:1010000021F07061154E766826F07066134F7E6091
:1010100012E000F48016B6F5801F06D1032606FA0A
:1010200005F4A14341F0706106E0460D360103FA74
:1010300006F6B14341F0706122B1460D360103FA64
:1010400006F6314300F00046B6F1004F02D1034EE0
:10105000F16101E0014E7160F0BD0000000001404F
:1010600041617047016170473EB55824684600F001
:101070000FF8002503E01DF8050044406D1C0C2D01
:10108000F9DB04B95824FF2C00D1852420463EBD4D
:101090000021064A00BF05E013780370401C521C73
:1010A0004B1CD9B20C29F7DB70470000E8F7FF1F93
:1010B0000948C0880849898808430749498808437E
:1010C000054909880843054908800846018804A0A5
:1010D00001F08AFE00BFFEE70000002008000020AB
:1010E0000D0A5B4846483D253034785D0D0A000006
:1010F0002DE9F043ADF6740D074688464FF0000920
:101100000DF60C0000F08CFA0025002417E02C49A5
:10111000601800F0A7FD064628466D1C03A90E5472
:10112000320A28466D1C0A54B5F5006F06D14FF4FB
:1011300000620DF60C0000F085FA0025A41CBC42EC
:10114000E5D32DB12A4603A90DF60C0000F07AFA7A
:101150000DF60C0000F0FCF93A461AA103A801F0C4
:1011600053FE00240BE00DF66400025D1AA101A8F5
:1011700001F04AFE01A903A8FFF71EF8641C102C19
:10118000F1DB17A103A8FFF717F803A800F0A4F9F3
:10119000002408E018F804100DF66400005D814298
:1011A00000D002E0641C102CF4DB00BF102C04DA29
:1011B00000200DF6740DBDE8F0830120F9E7000072
:1011C0000040000846696C6553697A653D256420D6
:1011D000204D44353D00000025303258000000000D
:1011E0000D0A000070B504460D46074884420AD136
:1011F0004FF480622946054800F07AFA06463146E7
:10120000024801F007FD70BD504354419221002077
:1012100070B504460548844207D1054800F09AFAA3
:1012200005462946024801F0F5FC70BD5043544183
:10123000922100202DE9F04FA1B08046444620685D
:101240007F49884208D020687E49884204D04FF008
:10125000FF3021B0BDE8F08F2079802802D06FF0F8
:101260000100F6E778A11DA801F0CEFDA11D1DA883
:10127000FEF7AEFF10B16FF00200EAE794F805A0A8
:10128000208B0190BAF1000F25D10198142802D0CB
:101290006FF00300DDE7C34610220BF11A016B4823
:1012A000FEF766FFD846DBF82A0069490860084661
:1012B000006810B96FF00400CBE7002065490860B2
:1012C0006549086065490860206862490968FFF758
:1012D00089FF0120BDE7BAF1020F7DD14746002604
:1012E00008E05A48815D07F11A00805D814200D014
:1012F00002E0761C102EF4DB00BF102E08DA58A096
:1013000000F0EAF82068FFF783FF6FF00500A0E720
:10131000D7F82E50D7F82A000290022D0CD34D4951
:1013200002980968884207D14A4800682918484845
:101330000068801C814208D94EA000F0CDF82068DA
:10134000FFF766FF6FF0060083E7AD1E2A4607F140
:101350003201002001F0B2FF814607F13200691C22
:10136000405C00021C9007F13200405D1C9908446B
:1013700080B21C901C9949450AD046A000F0ACF8F8
:10138000206834490968FFF72DFF6FF0070060E718
:1013900020682C4988420DD1002609E007F132006F
:1013A000805D42490978484007F132018855761C32
:1013B000AE42F3D307F1320229462648006800F016
:1013C000AFF826480068284424490860214800688E
:1013D00028442049086000E030E0204800681C49AB
:1013E0000968884210DB194919480068FFF780FE38
:1013F00040B92FA000F070F82068FFF709FF6FF0E8
:10140000080026E7002024E71248006864214843CA
:101410000F49096890FBF1F0034600900D482AA19E
:10142000026803A801F0F0FC03A800F055F820685A
:1014300008490968FFF7D6FE02200AE700BF08E75F
:10144000464F54415043544130000000DE0000201C
:10145000340000203C000020400000203800002024
:101460004D4435204D6F64696679215265444F21A2
:101470000D0A00004C656E677468206F72204F661D
:1014800066736574206572726F72215265444F21D4
:101490000D0A0000436865636B2043524320657268
:1014A000726F72215265444F210D0A002C000020FA
:1014B000436865636B204D4435206572726F7221FD
:1014C0005265444F210D0A004842443D25642025C1
:1014D0006425250D0A00000070B505462C460A203B
:1014E000FFF7DEFA0BA001F07FFC0BE021780B4840
:1014F00001F06BFA00BF4021084801F098F900287C
:10150000F9D0641C20780028F0D10A20FFF7C8FA2F
:1015100070BD00005B4941505D0000000038014093
:101520002DE9F04104460D461646002704F001005F
:1015300010B10020BDE8F081AAB20449601831461C
:1015400001F0FCFB80460120F4E7000000400008A9
:101550002DE9F04190B0044620680E9060680F902D
:101560002088C0F3C507382F02DAC7F1380001E040
:10157000C7F17800804642462849204600F062F8CC
:101580000026002518E004F11800E91C405C020662
:1015900004F11800A91C405C42EA004204F1180062
:1015A000691C405C42EA002004F11801495D0843CF
:1015B0004DF82600761C2D1D0E2EE4D3694604F14D
:1015C000080000F0CDFC0026002521E004F1080011
:1015D00010F8261050304155503830F82600C0F32E
:1015E000072204F15800691C4254503850F8260074
:1015F000C0F3074204F15800A91C4254503850F877
:101600002600000E04F15801EA1C8854761C2D1D9A
:10161000042EDBD310B0BDE8F0810000563700087F
:1016200000214160016005498160054AC260CA43EA
:101630000261034AD24342617047000001234567BB
:1016400089ABCDEF2DE9F04391B004460F46154626
:101650002088C0F3C509206800EBC50021688842D6
:1016600002D26068401C6060206800EBC50020600A
:10167000606800EB5570606033E017F8012B484656
:1016800009F1010904F118010A54B9F1400F28D1F8
:101690004FF0000800261AE004F11800F11C405C2D
:1016A000020604F11800B11C405C42EA004204F159
:1016B0001800711C405C42EA002004F11801895DA9
:1016C000084301A941F8280008F10108361DB8F1C6
:1016D000100FE1D301A904F1080000F041FC4FF024
:1016E0000009281EA5F10105C7D111B0BDE8F0839E
:1016F0002DE9F04104460E4617462546322128467C
:10170000FEF74FFD0F482860802028710220687185
:101710000DA1A81D01F078FB0C480088401C80B288
:101720000A490880E882182028831022084905F118
:101730001A00FEF71DFDC5F82A60C5F82E7032208C
:10174000BDE8F081504354413000000030000020DB
:10175000DE00002070B5044625462C212846FEF701
:1017600020FD0D48286080202871002068710BA1A1
:10177000A81D01F049FB0A480078E882122028835E
:1017800008A105F11A00FEF731FD00206885074920
:1017900008802C2070BD00005043544130000000F0
:1017A0002C0000204E554C4C000000003000002062
:1017B0002DE9F04104460E4617469846254650212D
:1017C0002846FEF7EEFC104828609520287104207A
:1017D00068710020E882362028830C4830F8160013
:1017E000A5F8460006EB460000EBC602084800EBF1
:1017F00082012C2205F11A00FEF7BAFCC5F84C80D4
:10180000AF645020BDE8F08150435441F6210020E0
:10181000B226002070B50446254622212846FEF750
:10182000C0FC0A48286095202871032068710020B8
:10183000E882082028835A20A883142068834FF464
:10184000FF10C5F81E00222070BD00005043544117
:1018500010B58CB016484068401E00EB400101EB0B
:10186000C0011348083000EB8100806A00F5805405
:101870000F484068401E00EB400101EBC0010C48DE
:10188000083000EB8100406A0444C4F30B00C0F54B
:10189000805004440748844201D30CB010BD064870
:1018A0000B9030222146684601F094FE00BFF4E719
:1018B000AA260020FFDF1F0012EFCDAB00BFFEE71E
:1018C0007047000070B5002100230F22C47804B3D4
:1018D000154C246804F4E064C4F5E064210AC1F105
:1018E0000403CA40447804FA03F184781440214385
:1018F00009010E4C0678A155047804F01F05012457
:10190000AC4005786D11AD0005F1E025C5F800414A
:1019100009E0047804F01F050124AC40044D06786A
:10192000761145F8264070BD0CED00E000E400E0C3
:1019300080E100E002490143024A11607047000063
:101940000000FA050CED00E004490978044A117022
:10195000024908700121034A5171704717000020A5
:10196000180000201000002008B50121084600F0F2
:1019700035F801211648FFF72BFB01211C2000F050
:101980002DF803208DF8020010208DF803000001CF
:10199000ADF8000069460F48FFF78EFA4FF400508B
:1019A000ADF8000069460C48FFF786FA4FF4005086
:1019B0000949086148208DF8030003208DF80200D2
:1019C0000820ADF8000069460248FFF775FA08BD27
:1019D00000023000000C01400010014029B1064A0D
:1019E00092690243044B9A6104E0034A926982437C
:1019F000014B9A61704700000010024030B5002191
:101A00000022002400232D4D6D6805F00C0121B14A
:101A1000042905D0082923D105E0294D056022E0DD
:101A2000284D05601FE0254D6D6805F47012234DAB
:101A30006D6805F48034022505EB92421CB9224DF5
:101A4000554305600BE01D4D6D6805F400351DB173
:101A50001E4D5543056002E01A4D5543056002E0F6
:101A6000174D056000BF00BF144D6D6805F0F00113
:101A70000909174D6B5C0568DD4045600F4D6D68C9
:101A800005F4E061090A124D6B5C4568DD40856034
:101A90000A4D6D6805F46051C90A0D4D6B5C4568CF
:101AA000DD40C560054D6D6805F44041890B094D69
:101AB0006B5CC568B5FBF3F5056130BD00100240F5
:101AC00000127A00001BB70000093D00808D5B000A
:101AD0008C0000209C000020F0B58BB0044600254F
:101AE00003E0334921F815506D1C6068A842F8D80E
:101AF000002656E006EB460101EBC60204F10801A0
:101B000001EB82002BA1FEF763FB002848D106EB16
:101B1000460000EBC60204F1080000EB82012C2213
:101B20006846FEF725FB374614E07A1C02EB4203B9
:101B300003EBC20304F1080202EB830107EB470247
:101B400002EBC70304F1080202EB83002C22FEF72C
:101B50000FFB7F1C6068401EB842E6D86168491ED2
:101B600001EB410202EBC10204F1080101EB82002A
:101B70002C226946FEF7FCFA354606E00C49681C43
:101B800031F8100021F815006D1C6068401EA84255
:101B9000F4D86068401E064A22F810600BB0F0BD11
:101BA000761C6068401EB042A4D800BFF6E7000073
:101BB000F62100207379732E696E690021B10288C5
:101BC00042F04002028004E002884FF6BF731A40E0
:101BD000028070470246002013890B400BB10120A0
:101BE00000E0002070470146888970478181704776
:101BF00010B50022028802F441520B884C8823431E
:101C00008C882343CC8823430C8923434C8923436A
:101C10008C892343CC8923431A430280838B4FF260
:101C2000FF74234083830B8A038210BD10B50446E2
:101C300000BF02210A48FFF7CDFF0028F9D0214656
:101C40000748FFF7D3FF00BF01210548FFF7C2FF98
:101C50000028F9D00248FFF7C6FFC0B210BD00004F
:101C600000300140014608887047704710B500F009
:101C700001F810BD0CB500200190009033480068B9
:101C800040F480303149086000BF3048006800F4FB
:101C9000003000900198401C0190009820B94FF648
:101CA000FF7101988842F0D12848006800F40030A4
:101CB00010B10120009001E0002000900098012860
:101CC00043D12348006840F01000214908600846CD
:101CD000006820F0030008600846006840F0020039
:101CE00008601A48406819494860084640684860DA
:101CF0000846406840F4806048600846406820F428
:101D00007C1048600846406840F4881048600846E7
:101D1000006840F08070086000BF0C48006800F068
:101D200000700028F9D00948406820F003000749F6
:101D300048600846406840F00200486000BF034821
:101D4000406800F00C000828F9D10CBD00100240DA
:101D50000020024000B587B002A8FFF74FFE0398AD
:101D6000009004A0DDE90423029901F03DF807B0DA
:101D700000BD0000535953434C4B3D25642C504348
:101D80004C4B313D25642C50434C4B323D25642C4B
:101D900048434C4B3D25640D0A00000030B5024617
:101DA0000B461946144607E008782578A84201D06A
:101DB000012030BD491C641C08780028F4D100BF04
:101DC000F7E7000010B500200F4908600F490860D0
:101DD0000F480078122806D0342805D0562807D09E
:101DE00078280ED107E00CE00A48FFF711FA08E066
:101DF000FEF738FB05E00848FFF76EFB01F08EFAAE
:101E000000BF00BF10BD0000200000201C0000200B
:101E10001700002050435441483700081448006818
:101E2000401C1349086001201249C870124800681C
:101E3000401C11490860322804DB002008600120A2
:101E40000C4908710D480078012804D10C4800782D
:101E5000401C0B4908700A480078012807DD012062
:101E60000849087003490870002004490870704749
:101E700084000020100000200C0000205C000020E6
:101E80005D0000205E00002010B51348006840F09F
:101E900001001149086008464068104908400E4991
:101EA0004860084600680E4908400B49086008462B
:101EB000006820F4802008600846406820F4FE0096
:101EC00048604FF41F008860FFF7D0FE4FF00060BD
:101ED0000449086010BD0000001002400000FFF837
:101EE000FFFFF6FE08ED00E010B517480068401C43
:101EF00020B115480068401C134908601348007859
:101F0000122806D034280CD056280BD0782818D1A7
:101F100009E00D480068012802D17820FFF714FD80
:101F20000FE00EE00DE008480068042800D210BD64
:101F30000548007800F0010010B105A0FFF7CCFAC9
:101F400000BF00BF00BFF2E7200000201700002004
:101F50004E6F20417070210D0A0000007047000094
:101F6000F0B505460C4628686968AA68EB6801EA7E
:101F7000020623EA01073E4327683E44FE4F3E44E3
:101F80003044C60146EA5060084400EA010622EAED
:101F900000073E4367683E44F84F3E4433441E0307
:101FA00046EA1353034403EA000621EA03073E43CB
:101FB000A7683E44F24F3E443244560446EAD232C9
:101FC0001A4402EA030620EA02073E43E7683E4459
:101FD000EC4F3E4431448E0546EA9121114401EA1A
:101FE000020623EA01073E4327693E44E64F3E448A
:101FF0003044C60146EA5060084400EA010622EA7D
:1020000000073E4367693E44E04F3E4433441E03AD
:1020100046EA1353034403EA000621EA03073E435A
:10202000A7693E44DA4F3E443244560446EAD2326F
:102030001A4402EA030620EA02073E43E7693E44E7
:10204000D44F3E4431448E0546EA9121114401EAC1
:10205000020623EA01073E43276A3E44CE4F3E4430
:102060003044C60146EA5060084400EA010622EA0C
:1020700000073E43676A3E44C84F3E4433441E0354
:1020800046EA1353034403EA000621EA03073E43EA
:10209000A76A3E44A6F524464F3E3244560446EA1B
:1020A000D2321A4402EA030620EA02073E43E76AF4
:1020B0003E44BB4F3E4431448E0546EA91211144D3
:1020C00001EA020623EA01073E43276B3E44B54F6F
:1020D0003E443044C60146EA5060084400EA010626
:1020E00022EA00073E43676B3E44AF4F3E44334411
:1020F0001E0346EA1353034403EA000621EA0307DA
:102100003E43A76B3E44A94F3E443244560446EA40
:10211000D2321A4402EA030620EA02073E43E76B82
:102120003E44A34F3E4431448E0546EA912111447A
:1021300001EA030622EA03073E4367683E449D4FD7
:102140003E443044460146EAD060084400EA0206B4
:1021500021EA02073E43A7693E44974F3E44334479
:102160005E0246EAD353034403EA010620EA01076C
:102170003E43E76A3E44914F3E443244960346EA6A
:1021800092421A4402EA000623EA00073E43276807
:102190003E448B4F3E4431440E0546EA1131114412
:1021A00001EA030622EA03073E4367693E44854F7E
:1021B0003E443044460146EAD060084400EA020644
:1021C00021EA02073E43A76A3E447F4F3E44334420
:1021D0005E0246EAD353034403EA010620EA0107FC
:1021E0003E43E76B3E44794F3E443244960346EA11
:1021F00092421A4402EA000623EA00073E43276996
:102200003E44734F3E4431440E0546EA11311144B9
:1022100001EA030622EA03073E43676A3E446D4F24
:102220003E443044460146EAD060084400EA0206D3
:1022300021EA02073E43A76B3E44674F3E443344C6
:102240005E0246EAD353034403EA010620EA01078B
:102250003E43E7683E44614F3E443244960346EABB
:1022600092421A4402EA000623EA00073E43276A24
:102270003E445B4F3E4431440E0546EA1131114461
:1022800001EA030622EA03073E43676B3E44554FCB
:102290003E443044460146EAD060084400EA020663
:1022A00021EA02073E43A7683E444F4F3E44334471
:1022B0005E0246EAD353034403EA010620EA01071B
:1022C0003E43E7693E44494F3E443244960346EA62
:1022D00092421A4402EA000623EA00073E43276BB3
:1022E0003E44434F3E4431440E0546EA1131114409
:1022F00081EA02065E4067693E443E4F3E443044F8
:10230000060146EA1070084480EA01065640276A32
:102310003E44394F3E443344DE0246EA53530344BD
:1023200083EA00064E40E76A3E44344F3E4432445E
:10233000160446EA12421A4482EA03064640A76B94
:102340003E442F4F3E443144CE0546EA51211144CC
:1023500081EA02065E4067683E442A4F3E443044AC
:10236000060146EA1070084480EA010656402769D3
:102370003E44254F3E4449E078A46AD756B7C7E8A3
:10238000DB702024EECEBDC1AF0F7CF52AC6874797
:10239000134630A8019546FDD8988069AFF7448B65
:1023A000BED75C892211906B937198FD8E4379A6FC
:1023B0002108B44962251EF640B340C0515A5E263A
:1023C000AAC7B6E95D102FD65314440281E6A1D8FE
:1023D000C8FBD3E7E6CDE121D60737C3870DD5F497
:1023E000ED145A4505E9E3A9F8A3EFFCD9026F679C
:1023F0008A4C2A8D4239FAFF81F6718722619D6DE0
:102400000C38E5FD44EABEA4A9CFDE4B3344DE021E
:1024100046EA5353034483EA00064E40E7693E44CC
:102420009F4F3E443244160446EA12421A4482EA5E
:1024300003064640A76A3E449A4F3E443144CE05C7
:1024400046EA5121114481EA02065E40676B3E4430
:10245000954F3E443044060146EA1070084480EA35
:102460000106564027683E44904F3E443344DE0206
:1024700046EA5353034483EA00064E40E7683E446D
:102480008B4F3E443244160446EA12421A4482EA12
:1024900003064640A7693E44864F3E443144CE057C
:1024A00046EA5121114481EA02065E40676A3E44D1
:1024B000814F3E443044060146EA1070084480EAE9
:1024C00001065640276B3E447C4F3E443344DE02B7
:1024D00046EA5353034483EA00064E40E76B3E440A
:1024E000774F3E443244160446EA12421A4482EAC6
:1024F00003064640A7683E44724F3E443144CE0531
:1025000046EA5121114461EA0306564027683E44D9
:102510006D4F3E443044860146EA9060084460EACC
:1025200002064E40E7693E44684F3E4433449E02F3
:1025300046EA9353034463EA01064640A76B3E44D0
:10254000634F3E443244D60346EA52421A4462EA9A
:1025500000065E4067693E445E4F3E4431444E058E
:1025600046EAD121114461EA03065640276B3E44F6
:10257000594F3E443044860146EA9060084460EA80
:1025800002064E40E7683E44544F3E4433449E02A8
:1025900046EA9353034463EA01064640A76A3E4471
:1025A0004F4F3E443244D60346EA52421A4462EA4E
:1025B00000065E4067683E444A4F3E4431444E0543
:1025C00046EAD121114461EA03065640276A3E4497
:1025D000454F3E443044860146EA9060084460EA34
:1025E00002064E40E76B3E44404F3E4433449E0259
:1025F00046EA9353034463EA01064640A7693E4412
:102600003B4F3E443244D60346EA52421A4462EA01
:1026100000065E40676B3E44364F3E4431444E05F3
:1026200046EAD121114461EA0306564027693E4437
:10263000314F3E443044860146EA9060084460EAE7
:1026400002064E40E76A3E442C4F3E4433449E020D
:1026500046EA9353034463EA01064640A7683E44B2
:10266000274F3E443244D60346EA52421A4462EAB5
:1026700000065E40676A3E44224F3E4431444E05A8
:1026800046EAD12111442E6806442E606E680E443D
:102690006E60AE681644AE60EE681E44EE60F0BD3B
:1026A000604BBBF670BCBFBEC67E9B28FA27A1EA72
:1026B0008530EFD4051D880439D0D4D9E599DBE6FF
:1026C000F87CA21F6556ACC4442229F497FF2A4324
:1026D000A72394AB39A093FCC3595B6592CC0C8FB4
:1026E0007DF4EFFFD15D84854F7EA86FE0E62CFE80
:1026F000144301A3A111084E827E53F735F23ABD6F
:10270000BBD2D72A91D386EB08B540F22551234896
:1027100000F09AF898B32248008810B901202149A6
:1027200008701E4800F04CF9C0B2009000201E490D
:1027300008701E480078E8B91948008841F2520133
:10274000884217DA9DF8000019491A4A12888854FD
:1027500018480088401C80B21649088041F2520196
:10276000884202DB0020134908800D480088401C85
:102770000B49088040F22551084800F034F8082140
:10278000064800F054F8012806D1044800F018F972
:102790000821024800F01EF808BD00000038014082
:1027A0005A0000205C0000205D0000201000002086
:1027B000EE000020580000207047704710B5FFF76A
:1027C000A3FF10BD10B5FFF7F7FF10BD10B5FFF761
:1027D000F4FF10BD01F40072B2F5007F00D100BF1C
:1027E000CA430280704710B50022002340F66A14E5
:1027F000A14200D100BF0A1201249440A3B2DC43DD
:10280000048010BD21B1828942F40052828104E02B
:1028100082894DF6FF731A40828170471AB1838A0C
:102820000B43838202E0838A8B4383827047024694
:102830000020B1F5007F00D100BF13880B400BB121
:10284000012000E00020704770B5024600240023FC
:102850000025002040F66A16B14200D100BFC1F346
:10286000421501F01F03012606FA03F3012D02D1E0
:102870009689334006E0022D02D1168A334001E0EA
:10288000968A33400C12012606FA04F41688344066
:1028900013B10CB1012000E0002070BDF0B503467B
:1028A000002400260025002040F66A17B94200D116
:1028B00000BF1846C1F3421401F01F06012707FAB2
:1028C00006F5012C01D10C3004E0022C01D11030AE
:1028D00000E014301AB107682F43076002E0076870
:1028E000AF430760F0BD00002DE9F04786B0054614
:1028F0000E460024A24600BFA1460027B08900B1C1
:1029000000BF2F462C8A4CF6FF700440F088044329
:102910002C82AC894EF6F3100440B088318908430C
:10292000718908430443AC81AC8A4FF6FF400440F0
:10293000B0890443AC8201A8FFF760F81F488742C2
:1029400002D1DDF810A001E0DDF80CA0A88900F4A8
:10295000004040B10AEBCA0000EB0A1031684900A0
:10296000B0FBF1F807E00AEBCA0000EB0A1031688F
:102970008900B0FBF1F86420B8FBF0F004012009F5
:10298000642101FB1089A88900F4004040B1322085
:1029900000EBC900B0FBF1F000F00700044308E0D1
:1029A000322000EB09106421B0FBF1F000F00F00C1
:1029B00004432C8106B0BDE8F087000000380140D8
:1029C00001468888C0F308007047C1F3080282807E
:1029D0007047000000B587B0012144F20400FEF703
:1029E000FDFF4FF40070ADF8140018208DF81700AB
:1029F00003208DF8160005A92548FEF75DFA4FF46F
:102A00008060ADF8140004208DF8170003208DF8C5
:102A1000160005A91E48FEF74FFA1E480190002037
:102A2000ADF80800ADF80A00ADF80C00ADF81000E4
:102A30000C20ADF80E0001A91748FFF755FF012142
:102A40001548FFF7DFFE4FF4E060FEF773FF252027
:102A50008DF8180000208DF819008DF81A0001205B
:102A60008DF81B0006A8FEF72DFF40210A48FFF74E
:102A7000B1FE002240F227710748FFF70FFF012245
:102A800040F225510448FFF709FF07B000BD0000E0
:102A900000080140105522000038014010B54048A0
:102AA000007812281BD13FA14248FFF777F930B9CF
:102AB0003420FEF749FF40A0FEF70EFD0EE042A1D4
:102AC0003C48FFF76BF930B95620FEF73DFF42A0B6
:102AD000FEF702FD02E045A0FEF7FEFC10BD304807
:102AE0000078342804D02E480078562800D0F5E726
:102AF0003048007850280BD12E484078432807D121
:102B00002C488078542803D12A48C078412800D026
:102B1000E4E72848007980281AD1364801882548FA
:102B2000FEF788FB044634B933A0FEF7D5FC5620E7
:102B3000FEF70AFFD2E714F1020F2EDA14F1060FA6
:102B40002BDD30A0FEF7C8FC7820FEF7FDFE24E068
:102B500018480079952820D1264801881548FDF7A6
:102B60008DFC04466CB9FEF773FEFDF7F3FB22A063
:102B7000FEF7B2FC7820FEF7E7FE0120244908703A
:102B8000ACE714F1020F08DA14F1060F05DD1DA001
:102B9000FEF7A2FC7820FEF7D7FE00BF9EE70000FC
:102BA00017000020444F574E4C4F41445F41505056
:102BB00000000000EE000020444F574E4C4F4144AF
:102BC0005F4150500D0A0000444F574E4C4F414456
:102BD0005F5246494C455300444F574E4C4F414479
:102BE0005F5246494C45530D0A0000002D2D2D2DF6
:102BF0000D0A000044000020436F6D706C65746521
:102C0000642100004941502053746F70210D0A0067
:102C10007000002070B505460E4600240BE0295DCB
:102C20000648FFF7D2FE00BF40210448FFF7FFFD32
:102C30000028F9D0641CB442F1DB70BD00380140BB
:102C400000BFFEE710B586B000F036F81021184836
:102C5000FEF708FA0020ADF804004FF48270ADF8DA
:102C600006000020ADF808000220ADF80A0001209F
:102C7000ADF80C004002ADF80E000020ADF81000D9
:102C8000ADF812000720ADF8140001A90948FEF7BD
:102C9000AFFF01210748FEF791FF4FF47A70FDF76F
:102CA00014FF00F04FFC0446012006B010BD0000E8
:102CB000000801400030014008B501210420FEF762
:102CC0008DFE01210803FEF789FE2020ADF80000EB
:102CD00003208DF8020018208DF80300694615487E
:102CE000FEF7EAF88020ADF8000069461148FEF7CB
:102CF000E3F84020ADF8000004208DF80300694699
:102D00000C48FEF7D9F81020ADF800008DF803004C
:102D100069460848FEF7D0F81020ADF800008DF89D
:102D2000030069460448FEF7C7F810210248FEF781
:102D300099F908BD00080140001001402DE9F04755
:102D400004460F469046B4F1006F02D31E488442F9
:102D500002D30120BDE8F087C4F3090008B10220C6
:102D6000F8E7FDF747FF3420FDF7D4FE6FF07F4012
:102D7000FDF74CFF2046FDF7D3FE0646042E01D09A
:102D80000320E7E76FF07F40FDF740FF002514E0E8
:102D9000795D681C385C01EB00201FFA80F960192E
:102DA0004946FDF707FF0646042E04D02246314669
:102DB00006A000F019F8A81C85B24545E8DBFDF730
:102DC000EFFE0020C6E7000000000408666C617397
:102DD000682D2D7374617475653D3D3D25642C250A
:102DE0006C750D0A000000000FB4054B10B503A967
:102DF000044A029800F02CF810BC5DF814FB0000A7
:102E0000F9320008C00000200FB4084B10B504A927
:102E100002AA039800F01CF8044602A9002000F062
:102E200048FA204610BC5DF814FB0000B3320008DD
:102E300002E008C8121F08C1002AFAD17047704783
:102E4000002001E001C1121F002AFBD170470000E1
:102E50002DE9FF4F8DB00F460546002606E02528D8
:102E60000BD0DDE90F1290476D1C761C28780028E6
:102E7000F5D111B03046BDE8F08F0024A246A1463E
:102E80000122EC4900E0044315F8013F203B02FA1F
:102E900003F00842F7D128782A2810D06FF02F02CB
:102EA0002878A0F13001092914D80AEB8A0102EB35
:102EB000410144F0020400EB010A6D1CF0E701CF70
:102EC0005FEA000A03D544F40054CAF1000A44F052
:102ED00002046D1C28782E2817D115F8010F44F034
:102EE00004042A280ED06FF02F022878A0F13001B8
:102EF00009290AD809EB890102EB410100EB01091C
:102F00006D1CF2E757F8049B6D1C28786C280FD0D5
:102F100006DC4C2817D068280DD06A2814D104E0AC
:102F2000742810D07A280FD10DE044F400140AE080
:102F300044F4801401E044F440146978814202D1E1
:102F400004F580146D1C6D1C2A786E2A1FD00CDCD1
:102F5000632A31D004DC002A8BD0582A11D1A3E097
:102F6000642A68D0692A0CD165E0732A2ED004DC6B
:102F70006F2A73D0702A04D19BE0752A6FD0782A0B
:102F80006ED01046DDE90F129047761C50E1C4F375
:102F90000250022806D0032809D0042801CF09D006
:102FA000066045E101CFF117C0E9006140E101CFC2
:102FB00006803DE106703BE117F8040B8DF8000038
:102FC00000208DF80100EB46012003E057F804BB18
:102FD0004FF0FF3061074FF0000102D40DE008F11F
:102FE0000101884649450FDA8045F8DB1BF80810D7
:102FF0000029F4D108E008F1010188468142FADB9A
:103000001BF808100029F6D1DDE90F23AAEB080010
:103010008146214600F036F9304400EB080604E012
:10302000DDE90F121BF8010B9047B8F10108F7D248
:1030300021464846F7E00A21C4F302534FF0000B43
:103040000891022B04D001CFC117032B09D00AE04D
:10305000FF1D27F00707F7E8020108E032E01FE054
:1030600020E000B2C117042B01D140B2C117031EEA
:1030700071F1000307DA4FF0000CD0EB0C006CEBA1
:1030800001012D2302E0230504D52B238DF82430E4
:10309000012303E0E30701D02023F7E7984658E037
:1030A0000A2110E010210EE010204FF0000B0890D4
:1030B0000CE010214FF0000B44F004044FF008091D
:1030C000089103E008214FF0000B0891C4F302536C
:1030D000022B04D001CF0021032B06D006E0FF1DF8
:1030E00027F00707F7E8020103E080B2042B00D1C4
:1030F000C0B24FF0000823072BD5702A07D0DDF8A7
:1031000020C08CF0100C5CEA0B0C05D00EE04023C4
:103110008DF82430012308E050EA010306D0302363
:103120008DF824308DF8252002239846DDF820C044
:103130008CF0080C5CEA0B0C0BD150EA010301D1B6
:10314000630706D530238DF824304FF00108A9F12C
:103150000109582A04D038A20B9208AA0A920BE05F
:103160003AA2F9E75B46089AFDF749F80B9B9B5C8E
:103170000A9A521E0A92137050EA0102F2D10A987A
:10318000ADEB000000F1200B600702D524F4803481
:1031900001E04FF00109D94502DDA9EB0B0000E089
:1031A000002000EB0B0141440890AAEB010AE00368
:1031B00006D4DDE90F232146504600F063F80644AB
:1031C0004FF0000908E009A911F80900DDE90F1224
:1031D000904709F10109761CC145F4DBE0030CD5E9
:1031E000DDE90F232146504600F04CF8064404E088
:1031F000DDE90F1230209047761C0899481E089090
:103200000029F5DC08E00A980A990078491C0A911F
:10321000DDE90F129047761CBBF10001ABF1010B09
:10322000F1DC21465046DDE90F2300F019F8064491
:103230006D1C1BE609280100303132333435363736
:1032400038396162636465660000000030313233F2
:103250003435363738394142434445460000000092
:103260002DE9F041044600251E461746880404D483
:1032700005E039462020B0476D1C641EF9D528466C
:10328000BDE8F0812DE9F041044600251E46904638
:10329000C80301D5302700E02027880404D505E0C5
:1032A00041463846B0476D1C641EF9D52846BDE836
:1032B000F0810A68531C0B6010707047F0B5074628
:1032C0000C461546002606E014F8011B384600F0AF
:1032D00007F80746761CAE42F6D33846F0BD00002C
:1032E000024682EA0100C0B2024B33F8100080EAC5
:1032F000222070479637000870B504460D46E1B2AB
:103300000548FFF762FB00BF40210348FFF78FFA33
:103310000028F9D0204670BD0038014010B50248A1
:1033200000F004F810BD00000040000810B504468D
:10333000206817490840B0F1005F1ED1002240F21A
:1033400024411448FFF7AAFA002240F225511148FF
:10335000FFF7A4FA002240210E48FFF75FFA002091
:103360004FF0E021086160680B4908602068FCF7B5
:10337000E9FE09480068804708E006E007A0FEF77C
:10338000ABF84FF47A70FDF77AFBF7E710BD000059
:103390000000FE2F00380140480000204E6F204101
:1033A00070700D0A00000000FFF714FB354800683C
:1033B0006422B0FBF2F1B1F1807F01D301201DE066
:1033C00021F07F40401E4FF0E022506150170F2245
:1033D000002807DA13071D0E2B4B00F00F04241FE3
:1033E0001D5503E013071C0E284B1C5400BF002082
:1033F0004FF0E022906107201061002008B100BF6B
:10340000FEE7FEF7B1FAFFF71DFCFDF787FCFDF7BD
:103410002BFE1F4908701F480021016081808171C7
:103420001220FEF791FAFEF795FCFCF74DFF28E01D
:103430001848007868B1FFF731FB00201649088072
:10344000144908701549088041F252011448FCF7EC
:10345000A8FE1048407920B100200E494871FEF7BF
:10346000B1FC0C48C07820B100200A49C870FEF7B2
:1034700075FD0848007920B1002006490871FEF763
:1034800033FDD5E7A000002018ED00E000E400E0E7
:103490002C000020100000205A00002058000020BE
:1034A000EE00002010B50446240300F0EDF800F013
:1034B00087F810210B48FDF7D3FD2020FEF7B6FB5F
:1034C000C4F30740FEF7B2FBC4F30720FEF7AEFBE0
:1034D000E0B2FEF7ABFB10210248FDF7C3FD00F0A0
:1034E0006FF810BD000801402DE9F04105460C467B
:1034F000174610211248FDF7B3FD0B20FEF796FB8F
:10350000C4F30740FEF792FBC4F30720FEF78EFBDF
:10351000E0B2FEF78BFBFF20FEF788FB2870002649
:1035200005E0FF20FEF782FBA855701C86B2BE4264
:10353000F7DB10210248FDF795FDBDE8F0810000A2
:10354000000801402DE9F041002400250026002755
:1035500010210F48FDF784FD9F20FEF767FBFF2039
:10356000FEF764FB0546FF20FEF760FB0646FF20E2
:10357000FEF75CFB074610210548FDF773FD2804A4
:1035800040EA062040EA07042046BDE8F08100003A
:103590000008014010B5002410210848FDF760FD27
:1035A0000520FEF743FBFF20FEF740FB04461021F9
:1035B0000248FDF757FD204610BD000000080140FD
:1035C00010B500BFFFF7E6FF00F001000028F9D1B9
:1035D00010BD00002DE9F04781460F4616464FEA20
:1035E0001738C7F30B0ACAF58054A64200DC3446EC
:1035F00044E04FEA08314FF480522248FFF774FF4D
:10360000002508E00AEB05001E49085CFF2800D0F1
:1036100003E0681C85B2A542F4DB00BFA54216DAC0
:103620004046FFF73FFF002507E019F8050005EBCE
:103630000A01144A5054681C85B2A542F5DB4FEAD2
:1036400008314FF480520F4800F02EF804E0224673
:103650003946484600F028F8A64200D10FE008F1AC
:1036600001084FF0000AA1442744301B86B2B6F58A
:10367000805F02DD4FF4805400E03446B9E700BFBC
:10368000BDE8F0872A36002010B510210548FDF767
:10369000E7FC0620FEF7CAFA10210248FDF7E2FC1B
:1036A00010BD0000000801402DE9F04107460E461C
:1036B0001446F0B2C0F58075AC4200DC254612E03D
:1036C0002A463146384600F013F8AC4200D10BE0F0
:1036D0002F442E44601B84B2B4F5807F02DD4FF48A
:1036E000807500E02546EBE700BFBDE8F0810000F3
:1036F0002DE9F04106460C461746FFF7C5FF10219D
:103700001048FDF7ADFC0220FEF790FAC4F3074025
:10371000FEF78CFAC4F30720FEF788FAE0B2FEF752
:1037200085FA002504E0705DFEF780FA681C85B21A
:10373000BD42F8DB10210348FDF794FCFFF740FF82
:10374000BDE8F0810008014048532D4941502D56F5
:103750003130370D0A00800000000000000000003A
:103760000000000000000000000000000000000059
:103770000000000000000000000000000000000049
:103780000000000000000000000000000000000039
:103790000000000000000000C1C081C1400101C361
:1037A000C003800241C201C6C006800741C70005B0
:1037B000C1C581C4400401CCC00C800D41CD000FB7
:1037C000C1CF81CE400E000AC1CA81CB400B01C9D6
:1037D000C009800841C801D8C018801941D9001B10
:1037E000C1DB81DA401A001EC1DE81DF401F01DD2E
:1037F000C01D801C41DC0014C1D481D5401501D707
:10380000C017801641D601D2C012801341D30011D7
:10381000C1D181D0401001F0C030803141F100337E
:10382000C1F381F240320036C1F681F7403701F52D
:10383000C035803441F4003CC1FC81FD403D01FFB6
:10384000C03F803E41FE01FAC03A803B41FB003957
:10385000C1F981F840380028C1E881E9402901EB2D
:10386000C02B802A41EA01EEC02E802F41EF002DAF
:10387000C1ED81EC402C01E4C024802541E5002706
:10388000C1E781E640260022C1E281E3402301E155
:10389000C021802041E001A0C060806141A100639F
:1038A000C1A381A240620066C1A681A7406701A5AD
:1038B000C065806441A4006CC1AC81AD406D01AFB6
:1038C000C06F806E41AE01AAC06A806B41AB0069D7
:1038D000C1A981A840680078C1B881B9407901BB0D
:1038E000C07B807A41BA01BEC07E807F41BF007D2F
:1038F000C1BD81BC407C01B4C074807541B5007706
:10390000C1B781B640760072C1B281B3407301B1D4
:10391000C071807041B00050C190819140510193BD
:10392000C053805241920196C0568057419700552E
:10393000C19581944054019CC05C805D419D005FB5
:10394000C19F819E405E005AC19A819B405B019954
:10395000C059805841980188C04880494189004B2E
:10396000C18B818A404A004EC18E818F404F018DAC
:10397000C04D804C418C0044C18481854045018705
:10398000C047804641860182C04280434183004156
:10399000C181818040400000B8390008000000204B
:1039A000C4000000302E00087C3A0008C40000204B
:1039B0006C490000402E00080000000000000000DC
:1039C00000000000000000000000000000000000F7
:1039D00000000000000000000000000000000000E7
:1039E00000000000000000000000000000000000D7
:1039F00000000000000000000000000000000000C7
:103A000000000000000000000000000000000000B6
:103A100000000000000000000000000000000000A6
:103A20000000000000000000000000000000000096
:103A30000000000000000000000000000000000086
:103A40000000000000000000010203040102030462
:103A5000060708090204060800A24A040000000044
:103A6000000000000102030406070809000000002E
:0C3A70000000000000000000000000004A
:0400000508000131BD
:00000001FF
